:020000040000FA
:020000000528D1
:08000800442883160130850035
:10001000860104308700D7308100831281010130CE
:100020009000970141309F0083160E309F0083128D
:100030002A30A9000A30AA00AB00AC000330A800A7
:100040002E30AD004030AE007930AF002430B0002B
:100050003030B1001930B2001230B3000230B400B9
:100060007830B5000030B6001030B7007F30B800EF
:100070002330B9001E30920083169D3092008C14FC
:100080008312E0308B0043280C080C1996288C183A
:10009000EF280B080B1956280B302D078400000899
:1000A0008600851005118511542809000B11810166
:1000B000070807195F280A30AA00AB00AC008512B8
:1000C0008F018E01960195010530970083160C155E
:1000D00083120C111430A0008820A00B6C281F156F
:1000E0001F1970281E08A1000530A200A10CA20B48
:1000F000762821080739363EA1000230A4007C3062
:10010000A5000000A50B8128A40B7F288516552883
:1001100010308700902087018D288E28000008006D
:100120009128922893289428000008000C11A60119
:10013000A7019701210895020319A7280318A128F0
:10014000B0280130A607031C9A28A70A9A28160887
:10015000031DA1280130A607031CB928A70AB92846
:100160001608031DB428B9289603FF309507950A91
:10017000A128AA01AB01AC016430A6020319C5286D
:100180000318C328CA28AC0ABC282708031DC328A3
:10019000AC0AD5282708031DD0286430A607D52827
:1001A000A703FF30A607A60AC3282C08093C031999
:1001B000E0280318E0280A30AA00AB00AC0055285C
:1001C0000A30A6020319E7280318E728E928AB0A32
:1001D000D5280A30A607EC282608AA0055288C1036
:1001E0002808A300A30BF8288514051585110129FB
:1001F000A30BFE2885140511851501298510051509
:10020000851528032907840000082D0784000008AD
:0C0210008600A80B55280330A8005528D4
:00000001FF
